:100000000C94B7020C94D4020C94D4020C94D40235
:100010000C94D4020C94D4020C94D4020C94D40208
:100020000C94D4020C94D4020C94AA230C947C2437
:100030000C947B1E0C94D4020C94D4020C94D40225
:100040000C94D4020C94D4020C94D4020C94D402D8
:100050000C94D4020C94031F0C94D4020C94D4027C
:100060000C94D4020C94D4020C94D4020C94D402B8
:100070000C94D4020C94D4020C94D4020C94D402A8
:100080000C94D4020C94D4020C94D4020C94D40298
:100090000C94D4020C94D4020C94D4020C94D40288
:1000A0000C94D4020C94D4020C94D402CA08CA084A
:1000B000F808F8085C097E099B0AFF0A8909240AE6
:1000C000360A360AA70ACA0AAF0AB20ABD0AB70A2E
:1000D000C20AE92410250826102508265C257F255C
:1000E0000826D625E525000B000A000900080007B0
:1000F0000006000500040003000200010000010BDF
:10010000010B0109010801070106010501040103B2
:10011000010201010100020B020C020902080207A0
:100120000206020502040203020202010200030B9E
:10013000030D030903080307030603050304030370
:10014000030203010300040B040E0409040804075E
:100150000406040504040403040204010400050B5E
:10016000050F05090508050705060505050405032E
:1001700005020501050068616E6477697265642F88
:1001800064616374796C2F64656661756C7420407A
:1001900020302E31352E32312D33382D67646136C3
:1001A000383038002E001E001F00200021002200E1
:1001B000230024002500260027002D004C001400F9
:1001C0001A000800150017001C0018000C0012008F
:1001D000130031002A0004001600070009000A007D
:1001E0000B000D000E000F0033423468E1001D616A
:1001F0001B00060019000500110010003600370032
:100200003861E50035413400E10450004F00000042
:100210000000520051002F0030000158E3004D0053
:100220002A002C004A00656429614B0028002B003D
:100230004E00E600A85D3A003B003C003D003E0059
:100240003F004000410042004300440001001E0204
:100250001F022F0230023102520024002500260026
:100260002502450001002002210226022702350056
:1002700051002100220023002E0201000100220271
:1002800023022F003000350224021E001F00200030
:1002900031000100005C01000100010001000000CC
:1002A00000000100370027002E00010001000100BE
:1002B0000100010001000100010001000100010036
:1002C0000100010001000100010001000100010026
:1002D0000100010001000100010001000100010016
:1002E0000100ED000100010001000100010001001A
:1002F0000100010001000100EF00EE00F00001002C
:1003000001000100010001000100AE000100010038
:10031000010001000100010001000100AC00AB0080
:1003200001000100010001000100F100F2000000E5
:100330000000A900AA00A8000100010001000100BE
:10034000010001000100010001000100B6000100F0
:100350000100010000000000000000002A2B28001E
:100360000000000000000000000000000000002964
:10037000000000002C1E3420212224342627252EA4
:10038000362D3738271E1F202122232425263333DC
:10039000362E37381F0405060708090A0B0C0D0E08
:1003A0000F101112131415161718191A1B1C1D2FD4
:1003B0003130232D350405060708090A0B0C0D0EF4
:1003C0000F101112131415161718191A1B1C1D2FB4
:1003D0003130354C0000000000000000000000003B
:1003E000000000000000000000000000000000000D
:1003F00000000000000000007E0F00D4FFFFFFC7D8
:10040000000000780E03440061006300740079006E
:100410006C0000001003410064006500720065007C
:100420007400680000000403090409023B00020193
:1004300000A0FA09040000010301010009211101D3
:1004400000012240000705810308000109040100A2
:10045000010300000009211101000122B600070577
:1004600082032000011201000200000008EDFE08D6
:100470001301000102000105010902A10185020921
:1004800001A1000509190129081500250195087524
:100490000181020501093009311581257F95027519
:1004A00008810609381581257F95017508810605A3
:1004B0000C0A38021581257F950175088106C0C098
:1004C00005010980A101850319012AB7001501263C
:1004D000B700950175108100C0050C0901A10185C7
:1004E0000419012AA002150126A0029501751081A8
:1004F00000C005010906A1018506050719E029E7E5
:10050000150025019508750181020507190029EFDD
:100510001500250195F075018102050819012905CD
:10052000950575019102950175039101C0050109B9
:1005300006A101050719E029E715002501950875B1
:100540000181029501750881010507190029FF1530
:100550000026FF0095067508810005081901290588
:10056000950575019102950175039101C000112453
:100570001FBECFEFDAE0DEBFCDBF11E0A0E0B1E0FB
:10058000E6E7FDE402C005900D92AE39B107D9F758
:1005900022E0AEE9B1E001C01D92A03FB207E1F751
:1005A0000E94DD150C94B9260C94000090E0FC012B
:1005B000E35EFE4F2081211118C0FC01E75DFE4F74
:1005C0008081E82FE295EF70F0E031A1282F2F70A5
:1005D00081E090E001C0880F2A95EAF7982F909566
:1005E000932391A392A1892B82A3089508950C943B
:1005F000F6020C94F7020C94F6020F931F93CF931C
:10060000DF9300D000D0CDB7DEB78091A00181117B
:100610000BC00E949B1B2FEF83ED90E32150804085
:100620009040E1F700C000008091D502882319F1C5
:100630001B828091D5028C8319828A8304E610E0A4
:1006400022E030E0AE014D5F5F4F60E080E40E9449
:100650009C1C8093D402811121C004E610E022E0AA
:1006600030E0AE014F5F5F4F6CE080E40E949C1C65
:100670008093D40213C0E7E1F1E041E050E09A0139
:10068000019002C0220F331F0A94E2F7822B21E06F
:10069000ED31F207A1F78093D502CACF0F900F90EA
:1006A0000F900F90DF91CF911F910F910895CF93ED
:1006B0000E94FD02C0E08C2F0E94D602CF5FCC309A
:1006C000D1F7A5E3B1E041E050E08D91E82FE2954C
:1006D000EF70F0E021A18F70BA0102C0660F771FA2
:1006E0008A95E2F7CB01962F9095922391A392A140
:1006F000892B82A371E0AB33B70739F7EEEAF1E05B
:10070000A2EAB1E08AEB91E0119211921D921D9242
:100710008E179F07C9F7CF910C9490053F924F9287
:100720005F926F927F928F929F92AF92BF92CF9281
:10073000DF92EF92FF920F931F93CF93DF9300D03E
:10074000CDB7DEB78091D402882349F08091A10112
:100750008F5F8093A101811102C00E94FD028DE193
:10076000482E81E0582E99E2A92E91E0B92EE12C75
:10077000F12CCC24C394D12C332433949E2C1A8294
:100780008E2CF20181912F018823D1F08091D40227
:1007900081112CC0C6010E2C01C0880F0A94EAF703
:1007A0008095898304E610E021E030E0AE014F5FE0
:1007B0005F4F62E180E40E949C1C8093D40216C0CB
:1007C000F5018081E82FE295EF70F0E021A18F70B4
:1007D000A60102C0440F551F8A95E2F7CA01922F65
:1007E000982B91A392A18095892382A350EA5A95D0
:1007F000F1F785E0891528F18091D402811172C04A
:1008000004E610E021E030E0AE014E5F5F4F63E1AF
:1008100080E40E94C91C8093D4028A8180958A83D7
:100820006A80712CA60102C0440F551F8A94E2F71A
:100830008A0100951095E2EAF1E080E090E0812CD9
:1008400034C0E5E3F1E020E030E04191A42FA2952F
:10085000AF70B0E090968C9190E04F7002C095958B
:1008600087954A95E2F780FD09C04A81C601022EAC
:1008700001C0880F0A94EAF7842B8A832F5F3F4FC9
:100880002630310511F7CCCFB90160237123718374
:10089000608332966D917C912617370711F088247A
:1008A000839401968630910581F0DF0120813181AA
:1008B000B301082E02C0759567950A94E2F760FFB0
:1008C000E3CFB901642B752BE2CF892D0E94D602AC
:1008D000882041F03092BA010E94DC1E9093BC0146
:1008E0008093BB01EFEFEE1AFE0AFFEFAF1ABF0ACB
:1008F0004CE0E416F10409F041CF8091BA0188235D
:10090000B9F08091BB019091BC010E94F41E409708
:1009100078F0E2EAF1E0AEEAB1E08EEA91E021910E
:1009200031912D933D938E179F07C9F71092BA010D
:100930000E94920581E00F900F90DF91CF911F915F
:100940000F91FF90EF90DF90CF90BF90AF909F906E
:100950008F907F906F905F904F903F900895E82F19
:10096000F0E0EE0FFF1FE255FE4F80819181089568
:100970000895883A9D4551F4FB018281882339F01E
:1009800086E791E00E94D80680E0089581E008950E
:100990009C013A9521153F4130F5BC0166277270E4
:1009A000AC01442754709C012227387094FF0FC07B
:1009B00090FF02C080E101C080E0672B09F08062F7
:1009C000452B09F08064232B79F080680895892FE6
:1009D0008170672B09F08260452B09F08460232B1E
:1009E00019F08860089580E00895CF93DF93EB01BC
:1009F0000E94C804FE01DF91CF910994CF93DF9349
:100A0000EC01805E9109089710F0209719F469E7CE
:100A100078E002C068E87BE0CE010E94F5048C2FEC
:100A2000DF91CF910C94CF07CF93DF93EC010E941D
:100A30002508CE01805E9109089710F0209719F4DF
:100A400060E878E002C06FE87BE0CE01DF91CF91F3
:100A50000C94F504CF93DF93EC010E94FE04C9339C
:100A6000D10549F42FEF87EE93E02150804090406C
:100A7000E1F700C00000CE01DF91CF910C94140586
:100A800081E008950C94B90408950C9444051F93D3
:100A9000CF93DF9300D000D01F92CDB7DEB749834C
:100AA0005A836B833091CA0189819A81311114C0B4
:100AB000662359F0222349F00E945B0D182F682FFE
:100AC00089819A810E94040D03C00E942F0D182F66
:100AD00069817A81812F04C00E945B0D69817A81CE
:100AE0000F900F900F900F900F90DF91CF911F916B
:100AF0000C94BB14FC01262F4081518162817381CB
:100B000084810C94470581E00895CF93DF93EC0135
:100B100060E00E947A05BE01DF91CF910C944505FB
:100B20000C94F9020C94FB0208950E94AE0B0E94F3
:100B300094052FEF84E39CE0215080409040E1F742
:100B400000C000000C94291F0F931F93CF93DF93D5
:100B50008C0161E00E947A05EC01B8010E94420517
:100B6000882309F444C0B801CE010E943F198823AC
:100B7000F1F1B801CE010E94491B8823C1F1B801EF
:100B8000CE010E945D19882391F1B801CE010E9427
:100B9000A51A882361F1F8018281882309F1CB35F8
:100BA0008DE5D807C1F050F4C115FCE5DF0781F0F1
:100BB000CF3DDC45A9F40E94B71219C0CC35EDE554
:100BC000DE0761F0CD35DD4559F40E94001208C002
:100BD0000E9495050CC00E94091202C00E940C12CE
:100BE000C801DF91CF911F910F910C94400580E0D7
:100BF000DF91CF911F910F9108950E945D1E0C947B
:100C0000F6060E94F9060C94631EDF92EF92FF92A3
:100C10000F931F93CF93DF93E82FF0E0EC5AFC4F34
:100C2000D490282F26952695269530E0F901EC5092
:100C3000FC4F0491877010E0082E02C015950795AF
:100C40000A94E2F701701127F901EC51FC4FE4908E
:100C5000F12C082E02C0F594E7940A94E2F791E093
:100C6000E922FF24F901EC52FC4FC491D0E002C00C
:100C7000D595C7958A95E2F7C170DD270115110555
:100C800019F081EE0E94CF07E114F10419F086EE0D
:100C90000E94CF078D2D0E947008EF2819F086EE74
:100CA0000E942508012B19F081EE0E942508CD2B0A
:100CB00051F08CE2DF91CF911F910F91FF90EF9057
:100CC000DF900C947008DF91CF911F910F91FF90EE
:100CD000EF90DF900895EF92FF920F931F93CF93C1
:100CE000DF938C01F62E8AE0E82EF80184918823A8
:100CF00009F457C0813009F042C0E8012196FE0195
:100D00008491813031F42196FE0184910E94700813
:100D100039C0823039F4E8012296FE0184910E94A4
:100D2000CF0730C0833039F4E8012296FE01849168
:100D30000E94250827C0843029F5E8012296FE018B
:100D4000249180E090E030E0205331092A303105D1
:100D500060F4E89EA001E99E500D1124C901840FA2
:100D6000951F2196FE012491EECF009759F0EFE9EF
:100D7000FFE03197F1F700C000000197F6CF0E9425
:100D80000506E8018E010F5F1F4F8F2D882309F4A0
:100D9000ACCFEFE9FFE03197F1F700C000008150E0
:100DA000F5CFDF91CF911F910F91FF90EF900895B4
:100DB00060E00C946B06982F9F709A50963010F05C
:100DC000805D01C0895A0C94050608950C94E506CF
:100DD00081E008950C94E8060895CF93C82F0E94EF
:100DE000E6068C2F0E94EA06CF91089580E00C94CD
:100DF000ED060E941F1D0C94ED060E941F1D909190
:100E0000BD01891721F08093BD010C94ED06089572
:100E1000DC0111962C9111979C91492F50E061E0D3
:100E200070E0FB0102C0EE0FFF1F9A95E2F7CF01C1
:100E300012966C91129730E0662329F06091CC01F4
:100E4000662361F10BC0F901EE0FFF1FE254FE4F64
:100E50006081718168237923672B01F16CE0629FC7
:100E6000F001639FF00D11244E0F5F1F440F551FBB
:100E7000FA01E951FF4FE4911196EC931197FA01B1
:100E8000EA51FF4FE491EC93220F331FF901E25432
:100E9000FE4F20813181822B932B0BC0220F331FF9
:100EA000F901E254FE4F8095909520813181822393
:100EB0009323918380830895CF93DF93CDB7DEB7DB
:100EC0002B970FB6F894DEBF0FBECDBF4F83588768
:100ED00069877A878B8761110E944C119F81888571
:100EE0002A853B85232B31F08F3F31F481E09F3FF2
:100EF00019F403C081E001C080E080FD04C0CE0190
:100F000007960E9408079E012F5F3F4F86E0F90178
:100F100011928A95E9F785E0FE013796D901019093
:100F20000D928A95E1F789819A814C815D81452BEB
:100F300031F09F3F31F491E08F3F19F403C091E00D
:100F400001C090E090FF09C049815A816B817C818A
:100F50008D819E810E94421005C0C9010E948305B7
:100F60008111F2CF2B960FB6F894DEBF0FBECDBF26
:100F7000DF91CF910895FC01808191810E949D0DA8
:100F800092959F70963051F4863F41F08091CC014C
:100F900091E089278093CC019093CB010895CF9362
:100FA000882309F450C0C82F8CEF8C0F813AD0F4FD
:100FB0006C2F80910201909103010E94981D88235B
:100FC00049F06C2F80910201909103010E94231E31
:100FD0000E946E116C2F80910201909103010E947A
:100FE000181E0CC080E28C0F883058F4C77081E066
:100FF00001C0880FCA95EAF70E942C11CF910C947A
:101000006E11EBE5EC0FE33040F4F0E0E759FE4FF2
:10101000808190E0CF910C94561DE8E5EC0FE7310C
:1010200050F4F0E0EE0FFF1FE55CFE4F80819181F0
:10103000CF910C946C1DCD3E30F08C2F0E94621627
:10104000CF910C943417CF910895882389F19CEFA8
:10105000980F913A40F4682F80910201909103011A
:101060000E94231E0DC090E2980F983058F48770AC
:1010700091E001C0990F8A95EAF7892F0E943211F9
:101080000C946E119BE5980F933020F480E090E073
:101090000C94561D98E5980F973120F480E090E06D
:1010A0000C946C1D8D3E20F00E94BD160C943417DC
:1010B00008951F93CF93DF93182FEB010E94CF0762
:1010C000209741F08FE99FE00197F1F700C0000001
:1010D0002197F6CF812FDF91CF911F910C94250896
:1010E000893319F060E070E002C060E570E00C94B4
:1010F0005908882321F00E942C110C946E11089538
:10110000882321F00E9432110C946E1108958F9261
:101110009F92AF92BF92CF92DF92EF92FF920F9386
:101120001F93CF93DF936C01C62F172FFC01D28141
:10113000058102950F700E9422118823D9F0DD23CA
:10114000C9F0812F807F803441F090E29C0F98306D
:1011500088F0803611F4C63F69F08091D70282FD95
:1011600009C082E00E94CE110E94221191E0E82E77
:10117000E92601C0E12CB12EB2949FE0B9228B2D5B
:1011800090E08C30910508F03AC2FC01EA5AFF4F1A
:101190000C946426012F0F70812F807F11F002952F
:1011A000007FDD2399F0002309F4B0C180E28C0FA9
:1011B000883010F0C11104C0802F0E942C1103C090
:1011C000802F0E943F110E946E11A0C18C2F0E949F
:1011D0002508002309F413C280E28C0F883010F038
:1011E000C11102C0802F29C0802F0E94451127C045
:1011F000912F9F70812F807FF92E803219F0F29409
:1012000080EFF822CC2319F0C130A1F13FC08091CA
:10121000D70282FF17C0DD2349F0FF2029F08F2D70
:101220000E942C110E946E1180E071C180E00E942A
:101230002508FF2009F4E3C18F2D0E9432110E947E
:101240006E11DDC1DD2371F0002341F0013031F476
:101250000E944F118F290E945711D1C10E944F1136
:101260008F290EC0002319F0013009F4C8C10E9473
:1012700064111EC0DD2339F0023008F0C0C18F2D8B
:101280000E947908BCC10111BAC112C0DD2319F056
:101290000023A9F33BC1002359F0C93309F047C12A
:1012A000FFEF27EE83E0F15020408040E1F73DC1A1
:1012B0008F2D0E948008A3C1812F8695869583700B
:1012C00019F0813071F09BC1DD2331F08C2F912F0B
:1012D00093700E94561D9BC180E090E00E94561DB5
:1012E0009FC1DD2331F08C2F912F93700E946C1DD4
:1012F0008EC180E090E00E946C1D92C18C2FDD2396
:1013000019F00E94621602C00E94BD160E94341796
:101310007EC1812F837009F048C0D11174C12C2F78
:10132000229526952770220F220F6C2F6F70862F23
:1013300090E0A0E0B0E0022E04C0880F991FAA1F21
:10134000BB1F0A94D2F7C4FF10C04FE050E060E02A
:1013500070E004C0440F551F661F771F2A95D2F70F
:10136000409550956095709503C040E050E0BA01FB
:10137000212F2695269523704A015B01882A992AF8
:10138000AA2ABB2AC501B401223049F058F4213001
:1013900019F00E941A0C37C10E94080C34C10E9437
:1013A0002C0C31C10E94060C2EC1DD2319F0812FB7
:1013B000817001C08695882309F425C12C2F2295C0
:1013C00026952770220F220F6C2F6F70862F90E0CA
:1013D000A0E0B0E0022E04C0880F991FAA1FBB1F17
:1013E0000A94D2F7C4FF10C04FE050E060E070E014
:1013F00004C0440F551F661F771F2A95D2F74095EA
:1014000050956095709503C040E050E0BA01212FDF
:101410002695269523704A015B01882A992AAA2AD3
:10142000BB2AC501B401223049F058F4213019F02B
:101430000E94DF0CE8C00E94CD0CE5C00E94F10CB8
:10144000E2C00E94400CDFC0012F0F70DD2339F095
:10145000802F0E94660C8C2F0E947908D4C08C2F9C
:101460000E948008802F0E94870CCDC0C23F19F1D6
:1014700028F4C03F41F0C13FB9F044C0C33F11F16F
:10148000C43F71F03FC0DD2339F00111B8C0812F96
:101490008F710E94AC0CB3C0023008F0B0C0F7CF1F
:1014A0008091D70282FF18C0DD2339F0812F8F7120
:1014B0000E94660CA4C0DD23C9F3812F8F710E94A6
:1014C000870C9DC0DD2329F0812F8F710E94510C64
:1014D00096C00E944C0C93C0DD2351F0012F0F7178
:1014E000802F0E94660C63E0802F0E94B31187C09A
:1014F00081E00E94CE11023008F481C082E00E9497
:10150000CE117DC0DD2331F0002381F28C2F0E94AB
:10151000CF0775C0002389F2C93349F42FEF87EE56
:1015200093E0215080409040E1F700C000008C2FF4
:101530000E94250864C08C2F90E0FC01E05FF10957
:10154000E730F10598F5EE59FF4F0C946426DD2342
:1015500009F466C09091CC0181E0892705C0D09341
:10156000CC0155C081E08D278093CC0150C0D111B2
:101570004EC081E08093CC0153C0D11148C010927D
:10158000CC014EC0DD2319F00E94FA1040C00E9429
:10159000061146C0DD2339F08091CB018823D1F2BA
:1015A0001092CB0134C00023A9F23AC08091CB0144
:1015B0000023C1F0882341F09091CC0181E089277C
:1015C0008093CC011092CB018C2FDD2319F00E9467
:1015D000CF071DC00E94250886E0F60111928A956A
:1015E000E9F71EC0882399F0D11111C09091CC0168
:1015F00081E089278093CC011092CB0111C088EF44
:101600008B0D843020F40E941F1D0E94ED06DD2307
:1016100039F0107F103611F4C63F11F00E941411FA
:10162000EE20E9F00E94F61080FD19C0F60112824A
:101630000E94F0100E94660CC6010E94540B0E948A
:10164000F010DF91CF911F910F91FF90EF90DF90FD
:10165000CF90BF90AF909F908F900C94870CDF91AC
:10166000CF911F910F91FF90EF90DF90CF90BF909F
:10167000AF909F908F9008950F931F93CF93DF9318
:10168000EC01688179818A810E94A80D8C010E94F9
:10169000030D0E94F40BB801CE010E948708DF9170
:1016A000CF911F910F910895CF93DF93EC01988113
:1016B00089812B813C81232B31F08F3F31F481E0F4
:1016C0009F3F19F403C081E001C080E080FD1DC090
:1016D000CE010E94A405811110C00E94221188230E
:1016E000A1F08A81882389F08091D70282FD0DC004
:1016F00082E0DF91CF910C94CE11CE010E943C0B81
:10170000CE01DF91CF910C948505DF91CF910895A3
:10171000882321F00E943F110C946E1108958823B4
:1017200021F00E9445110C946E11089580E090E024
:101730000E94561D80E090E00E946C1D0E944C119A
:101740000E946E110E9465180C943417809102015A
:10175000909103010E942E1E0C94960B0E943C1146
:101760000C94A60B92959F70963079F010F49250DD
:1017700001C09A50923068F4803F69F018F4883EB6
:1017800040F409C0843F29F406C0883E20F0813F20
:1017900011F080E0089581E00895FC01808191813D
:1017A0000E949D0D0E94B20B0895CF93DF9300D04D
:1017B00000D01F92CDB7DEB70F900F900F900F9013
:1017C0000F90DF91CF910895CF93DF9300D000D099
:1017D00000D0CDB7DEB726960FB6F894DEBF0FBEA9
:1017E000CDBFDF91CF910895089508950C94F50B26
:1017F0000C94F60B0E94F80B6093FE017093FF01AE
:1018000080930002909301020C94960B0C94FA0BB7
:101810000F931F930091FE011091FF012091000290
:1018200030910102602B712B822B932B1F910F9112
:101830000C94FA0B0F931F930091FE011091FF017E
:1018400020910002309101026023712382239323AF
:101850001F910F910C94FA0B0F931F930091FE01AF
:101860001091FF0120910002309101026027712741
:10187000822793271F910F910C94FA0B0C94F50B70
:101880000E943E0C6093FA017093FB018093FC016F
:101890009093FD010C94960B60E070E0CB010C94EA
:1018A000400C0F931F9341E050E060E070E08A012C
:1018B0009B0104C0000F111F221F331F8A95D2F70E
:1018C000C901B8011F910F910C94400C0F931F9305
:1018D00041E050E060E070E004C0440F551F661F17
:1018E000771F8A95D2F78091FA019091FB01A09120
:1018F000FC01B091FD018A019B01082B192B2A2BB9
:101900003B2BC901B8011F910F910C94400C0F9310
:101910001F9341E050E060E070E004C0440F551FA9
:10192000661F771F8A95D2F7409550956095709500
:101930008091FA019091FB01A091FC01B091FD0111
:101940008A019B01082319232A233B23C901B801DB
:101950001F910F910C94400C0F931F9341E050E0A6
:1019600060E070E004C0440F551F661F771F8A9522
:10197000D2F78091FA019091FB01A091FC01B09106
:10198000FD018A019B01082719272A273B27C90146
:10199000B8011F910F910C94400C0F931F9300916D
:1019A000FA011091FB012091FC013091FD01602BA7
:1019B000712B822B932B1F910F910C94400C0F9342
:1019C0001F930091FA011091FB012091FC013091CD
:1019D000FD0160237123822393231F910F910C94A7
:1019E000400C0F931F930091FA011091FB0120917D
:1019F000FC013091FD0160277127822793271F91F9
:101A00000F910C94400C08952CE0929F800D1124AE
:101A1000E82FE695E695E695877051E001C0550FF1
:101A20008A95EAF785E0E89FF0011124E353FE4F21
:101A300020E030E070E04081CB01022E02C096959C
:101A400087950A94E2F781708195842785238427FE
:101A500081932F5F3F4F2530310569F708952CE0C2
:101A6000929F800D1124682F669566956695982F34
:101A7000977085E0689FB001112440E050E080E05D
:101A8000FB01E40FF51FE353FE4F208130E0092EE8
:101A900002C0369527950A94E2F721703327042E69
:101AA00001C0220F0A94EAF7822B4F5F5F4F453047
:101AB000510531F70895BF92CF92DF92EF92FF92D6
:101AC0000F931F93CF93DF938C01C090FA01D090B6
:101AD000FB01E090FC01F090FD018091FE019091EE
:101AE000FF01A0910002B0910102C82AD92AEA2A76
:101AF000FB2ACFE1D0E0D701C6010C2E04C0B69579
:101B0000A795979587950A94D2F780FD04C02197F1
:101B100090F7B12C07C0BC2EB8018C2F0E94CE14B8
:101B20000197A9F38B2DDF91CF911F910F91FF901A
:101B3000EF90DF90CF90BF900895CF93DF93EC01AB
:101B40000E945B0DBE010E94CE14DF91CF910895DB
:101B50001F93CF93DF93EB019091CA01992321F05A
:101B6000CB010E949D0D13C0882349F0CB010E9438
:101B70005B0D182F682FCE010E94040D04C0CB010D
:101B80000E942F0D182FBE01812F0E94CE14DF91CD
:101B9000CF911F9108951F93CF93DF93C0910202BD
:101BA00016E080910302C81799F0D0E01C9FF00165
:101BB0001D9FF00D1124EC5FFD4F4081518162812A
:101BC0007381848195810E94E40B2196C770E9CFCF
:101BD000DF91CF911F9108954091340250913502C9
:101BE00060913602709137028091380290913902EB
:101BF0000C94E40BEF92FF920F931F93CF93DF931C
:101C00008091390282958F7009F065C0809136020B
:101C1000882309F460C080910202F09003021091C1
:101C2000340200913502609137027091380291E0E0
:101C30001F3F09F090E0C0910001D0910101292FD0
:101C400096E0E92E8F1509F446C06115710521F063
:101C50000F3F21F030E003C031E001C0322F90E0AF
:101C600030FD36C0E89EF001E99EF00D1124DF0141
:101C7000AC5FBD4F11963C911197301329C03C9138
:101C8000311326C012963C911297311121C0139640
:101C90004D915C911497461B570B4C175D07C0F490
:101CA000809139028F70806180933902E75FFD4F28
:101CB00080818F708061808384E392E00E94540B66
:101CC000DF91CF911F910F91FF90EF900C94CB0D6E
:101CD00001968770B7CFDF91CF911F910F91FF9041
:101CE000EF9008959F92AF92BF92CF92DF92EF92C2
:101CF000FF920F931F93CF93DF93CDB7DEB761971A
:101D00000FB6F894DEBF0FBECDBF8C0185E0F801A1
:101D1000DE011D9601900D928A95E1F7D801129689
:101D2000EC9090913402E09135022091370230918D
:101D300038022115310531F0EF3F31F481E09F3F4A
:101D400019F403C081E001C080E0B82FB1709B2E70
:101D500080FD47C1D8014C9111965C911197139663
:101D6000AD90BC90149784E3C82E82E0D82EF090FA
:101D70003602B501621B730B209100013091010105
:101D8000FF2009F4D9C0809139026217730708F067
:101D900095C0282F207F09F052C05E1313C049134D
:101DA00011C0FE2CE1100EC08F708061809339024B
:101DB0000E94EC0DC6010E94540B80913902F8017B
:101DC00085834DC1AB2831F05F3F31F481E04F3F57
:101DD00019F403C081E001C080E080FD03C081E010
:101DE0008E2502C080E090E0F82FF170FF2E80FF7A
:101DF0001CC0809102022091030236E0821709F490
:101E00000BC190E0389FF001399FF00D1124EC5F79
:101E1000FD4F6181561306C06081461303C0628185
:101E2000E61203C001968770E9CFFE2CEE2009F47C
:101E300016C18091390281608093390254C05E13CB
:101E400006C0491304C0E11002C0F80199C0C801DE
:101E50000E94CD0B882361F1EE2051F120913902CF
:101E6000822F82958F7090E0029774F080913402F7
:101E70009091350298878F831986BB86AA862C8716
:101E8000CE0107960E94540B86E0F801A4E3B2E06D
:101E900001900D928A95E1F70E94FA0D0E94EC0DD7
:101EA0000AC05E1711F1C8010E94CD0B81112CC030
:101EB000C8010E94540BFF24F394D1C0282F207F27
:101EC00081F77A2DB98AA88A6E2D89890E94D50B4F
:101ED00084E392E00E94540B86E0D6011D928A951D
:101EE000E9F70E94EC0DF12CBAC04913DCCFE110E8
:101EF000DACFF8018583C8010E94540B86E0D60131
:101F00001D928A95E9F7ABC0EE2091F2209139023B
:101F1000822F82958F7090E002970CF4B5CF80915C
:101F20003402909135029A8389831B82BD82AC82F0
:101F30002E83CE010196A6CF6217730708F044C026
:101F4000FE2CEE2009F4B4CF5E1330C049132EC02E
:101F50002091390220FD21C0822F82958F70482F59
:101F600050E041155105C9F0F80125834F30510566
:101F700041F08F5F982F9295907F822F8F70892BE1
:101F80008583C8010E94540B86E0F801A4E3B2E007
:101F900001900D928A95E1F73CC086E0F801A4E338
:101FA000B2E001900D928A95E1F759C0C8010E94F4
:101FB000CD0B811169CF8091390281608093390204
:101FC000C8010E94540B4BC07A2DB98AA88A6E2D85
:101FD00089890E94D50B86E0D6011D928A95E9F782
:101FE00018C0EE2009F464CFC8010E94CD0BF82E72
:101FF000882309F45DCF86E0F801A4E3B2E0019004
:102000000D928A95E1F784E392E00E94BB070E945B
:10201000FA0D0E94EC0D23C04D875E878D859E854D
:102020000E949D0D292F22952F70223028F49F7039
:1020300039F0811105C00BC0243028F49F7049F499
:10204000805E883020F0C8010E94540B9F2CF92C30
:1020500006C0D80115969C91907F91F7F8CF8F2DEF
:1020600061960FB6F894DEBF0FBECDBFDF91CF9162
:102070001F910F91FF90EF90DF90CF90BF90AF90A6
:102080009F9008951F93CF93DF93CDB7DEB72C9722
:102090000FB6F894DEBF0FBECDBF4F835887698758
:1020A0007A878B879C87CE0107960E94720E8823C1
:1020B000D1F09F8188852A853B85232B31F08F3F86
:1020C00031F481E09F3F19F403C081E001C080E05A
:1020D00080FD47C04F81588569857A858B859C85B1
:1020E0000E94E40B3EC086E0FE013796DE011196A9
:1020F00001900D928A95E1F7FF81E8856A857B85DD
:102100006115710531F0EF3F31F481E0FF3F19F4C3
:1021100003C081E001C080E080FD23C02091030264
:1021200030E0C9010196877099274091020250E082
:1021300084179507F1F1F983EA837D836C8396E038
:10214000929FD001939FB00D1124AC5FBD4FFE0153
:10215000319601900D929A95E1F7809303020E94C7
:10216000CB0D16E08091020290910302891771F164
:10217000189FC00111248C5F9D4F0E94720E88230E
:1021800029F1E09102021E9FF0011124EC5FFD4F46
:102190004081518162817381848195810E94E40B29
:1021A0008091020290E00196877099278093020245
:1021B000D9CF0E94AE0B1092030210920202E4E308
:1021C000F2E086E0DF011D928A95E9F72C960FB6C2
:1021D000F894DEBF0FBECDBFDF91CF911F91089560
:1021E00080915B02859585958595089580915B0228
:1021F0008770089582E080935A0281E08093CC0139
:10220000089510925A021092CC01089580915A02BA
:10221000823019F481E080935A0280915A0283300F
:1022200011F40C940111089580915A02823019F42E
:1022300083E080935A0280915A02813011F40C9409
:102240000111089590915B02977081E009F480E09C
:10225000089580917E02089590917E02892B80934B
:102260007E020895809590917E02892380937E025C
:10227000089580937E02089510927E0208959091B1
:102280007D02892B80937D020895809590917D0237
:10229000892380937D02089510927D020895809194
:1022A0005C02089508950C9452110C94531190916E
:1022B000D70292FD08C090915C02981721F080939C
:1022C0005C020C945511089580915C02882329F0DA
:1022D00010925C0280E00C9455110895CF93DF9327
:1022E000E0910201F091030180917E028083E091F0
:1022F0000201F0910301908180917D02892B8083FE
:1023000080915C02882381F0E0910201F091030149
:102310009081892B808380910201909103010E941A
:10232000821D81110E946411C0910201D0910301AC
:1023300040E250E06AE372E0CE010E946A26892BF7
:1023400069F080E2FE01AAE3B2E001900D928A9565
:10235000E1F7CE01DF91CF910C942E1DDF91CF914B
:1023600008950C9452119091D70292FD10C098E0FC
:10237000899F90011124262B20935B020E94660CFA
:1023800080915B028595859585950C94B1110C948F
:10239000660C10925B0280E00C94B11120915B02FC
:1023A0008095822380935B02982F977099F430E098
:1023B000482F082E000C550B2417350759F0909123
:1023C000D70292FD07C08595859585950E94870C5B
:1023D0000C94C91108959091D70292FB222720F9FD
:1023E000281769F080FB92F99093D7028091D6026A
:1023F0009091D7020E94331282E00C94CE1108957E
:102400008091D70282FB882780F991E089270C947C
:10241000EB1181E00C94EB1180E00C94EB1180E067
:1024200090E00E947F2621E0893E9E4F09F020E047
:10243000822F089582E090E00C94772683E090E06C
:102440000C947726CF9384E090E00E947726C82FE3
:1024500082E290E00E9477262C2F30E0A901582BD1
:10246000CA01CF910895CF93C92F682F84E090E0DF
:102470000E9485266C2F82E290E0CF910C948526F5
:10248000AB01BC018FE090E00C949726AB01BC013E
:1024900083E190E00C94972660E070E0CB010C940F
:1024A000461260E070E0CB010E9440120C944C1286
:1024B00069EE7EEF80E090E00E94A32660E082E07B
:1024C00090E00E94852660E083E090E00E948526EF
:1024D0001092FE011092FF01109200021092010270
:1024E00060E084E090E00E94852660E082E290E077
:1024F0000E94852660E085E090E00E94852660E0ED
:1025000086E090E00E9485266FEF87E090E00E94D1
:10251000852640E050E0BA0188E090E00E949726CE
:1025200060E08DE090E00E94852640E050E0BA0136
:1025300088E190E00E94972660E087E190E00E94A9
:10254000852640E050E0BA018CE190E00E94972699
:1025500060E070E080E290E00E94A32640E050E05E
:10256000BA0188E190E00E9497260C9451120C94D5
:102570005812682F8EE090E00C9485260E94E81E89
:1025800060938F02709390028093910290939202D5
:1025900060938B0270938C0280938D0290938E02D5
:1025A000089585B7806885BF85B7806885BF089521
:1025B00081E008950C94D81208950C94DC120C94C8
:1025C000DC120C94DF120C94DC120C94E3120C94C9
:1025D000DC120E94D1128AEA95E10E94151D0E9428
:1025E000E7120C94E5120E94DD120C94DC120E949A
:1025F000AD150E94EC060C949B180E94D31E0E94FD
:1026000057030E94F7120C94E1125F926F927F922F
:102610008F929F92AF92BF92CF92DF92EF92FF92F2
:102620000F931F93CF93DF93CDB7DEB72A970FB6E3
:10263000F894DEBF0FBECDBF0E948E03C82E81115D
:102640000E94BE123FE7832E32E0932E00E010E09E
:10265000502E802F0E94AF045C01F40161907190B4
:102660004F016826792661147104B1F40F5F1F4F82
:102670000630110569F78FEF89838A831B820E94D8
:10268000DC1E8160782F9D838C8349815A816B8108
:102690008D810E945C073AC08091930281FD0E9467
:1026A000B804D12CEE24E394F12CC3018E219F2198
:1026B000892B29F10E94DA128823A9F0DE825F8239
:1026C000AE20BF2081E0AB2809F480E088870E941B
:1026D000DC1E8160782F9A8789874E815F816885AB
:1026E0008A850E945C07000F111FF801E158FD4F19
:1026F00080819181E826F926F182E08207C0D39497
:10270000EE0CFF1CFCE0DF12D0CFB0CF81E0C11097
:1027100001C080E02A960FB6F894DEBF0FBECDBF91
:10272000DF91CF911F910F91FF90EF90DF90CF90AD
:10273000BF90AF909F908F907F906F905F90089523
:102740000E9405130E9452170C94FD06CF93DF934D
:102750000E94D314EC01811522E5920708F04AC0CB
:10276000811531E5930708F0C2C0883E910528F530
:10277000803E910508F0FBC0883A910570F4853AD7
:10278000910508F089C08130910509F482C008F4F0
:10279000EBC0049708F0EBC0E7C08F3B910508F051
:1027A000E3C0C85AD0E0CC0FDD1FC459DE4F0990FA
:1027B000D881C02DCE019464DBC0811540E294071E
:1027C00058F4811551E0950708F0D1C08D3E910570
:1027D00008F4CAC09065CCC0C11580E4D80708F4DD
:1027E000C3C0C11520E5D20708F060C0DF70CE017C
:1027F000906ABEC0811536E5930728F5811545E539
:10280000940708F091C0811554E5950708F086C03B
:10281000AC0143705527282F26952695C115D34521
:1028200008F06BC081E090E002C0880F991F4A95C4
:10283000E2F740E2249F90011124EC01C22BD32B3C
:10284000CE019C6895C0811529E5920768F4811531
:1028500038E5930708F071C08115974508F084C0EA
:10286000DD27CE01906684C081155AE5950708F4EE
:102870006AC090568115904208F076C08D2F8F71F6
:102880000E946715DD27D0628F71AE01582BCA01F7
:102890006FC081E090E06CC0C55AD0E0C656DE4FF4
:1028A0008881C82FD0E0CE01906462C0CE0174E070
:1028B000969587957A95E1F7282F23703C2F3370F2
:1028C00081E090E002C0880F991F3A95E2F79C687A
:1028D000AC01522B9A019C2F9F709695969550E2D1
:1028E000959FE0011124C9018C2B9D2B41C0D82F4D
:1028F000CC27CE01816F906A3BC081E090E002C09E
:10290000880F991F4A95E2F750E2259F9001112404
:10291000EC01C22BD32BCE019A682AC0D82FCC272A
:10292000CE01846F906A24C00E9467158F7190E079
:10293000D82FCC27CE0190621BC0D82FCC27CE0138
:10294000806F906A15C08F700E94671594E0D695CD
:10295000C7959A95E1F7CF70D0E0DC2FCC27D069EE
:102960009E01282BC90104C080E090E001C0CE0187
:10297000DF91CF91089528E4829FC0011124FC01CA
:102980002CE0729FE00DF11D1124E60FF11DEE0FFA
:10299000FF1FEC55FE4F8591949108950E94BB1442
:1029A0000E94A61308958238910569F1B0F481332D
:1029B000910509F46DC048F48932910509F463C0AA
:1029C0008A32910509F469C008958533910509F4A7
:1029D00055C089339105B9F00895833E910569F199
:1029E00038F4803E9105B1F0823E910509F10895D9
:1029F000863E9105A9F1873E9105B9F1843E910586
:102A000009F064C023C02091D60220FD4FC021FDF3
:102A10004DC008958091D60280FD44C08091D702B8
:102A200080FF44C08091D60284FD42C083EE4DC039
:102A30008091D60282FF38C0F5CF8091D60282FD08
:102A400033C08091D70280FD31C0ECCF8091D70296
:102A500081FF32C08091D60284FD2AC087EE35C046
:102A60008091D60283FF26C0F5CF8091D60283FDE8
:102A700021C08091D70281FD1FC0ECCF8091D6028A
:102A800085FD1CC01DC08091D60285FD19C016C0F1
:102A90008091D60286FD16C017C08091D60286FDB1
:102AA00013C010C089E311C082EE0FC080EE0DC0CC
:102AB00080E00BC086EE09C084EE07C089E205C045
:102AC00085E303C08AE201C081E390E0089590911C
:102AD000D60292FF0DC0282F2871283019F4877F65
:102AE000846006C0282F2471243011F48B7F886005
:102AF00093FF0DC0282F2871283119F4877E846137
:102B000006C0282F2471243111F48B7E8861209116
:102B1000D70220FF0DC0382F3871383019F4877F65
:102B2000816006C0382F3171313011F48E7F88609A
:102B300021FF0DC0282F2871283119F4877E81616B
:102B400006C0282F2171213111F48E7E886194FDF9
:102B5000877E089580E0089508950E940F128111E4
:102B600002C00E94B7120E941A12809393020E9420
:102B700022129093D7028093D6020E94AC150E9435
:102B80001E12682F70E080E090E00E94060C6091B9
:102B9000FA017091FB018091FC019091FD010C9470
:102BA0003E0C0E9402210E94FD120C940E210E94F4
:102BB00012210E94A0130C942C210E947A1E0E94C4
:102BC000E9200E94E9120E94D1150E94D7150E94A7
:102BD000F312FBCF80919C0280FF06C06091080138
:102BE00070E0660F771F26C081FF04C06091080166
:102BF00084E005C082FF07C06091080188E0689FFB
:102C0000B001112417C090919B029923D1F06091DB
:102C10000701961788F72091080188E0289F900106
:102C20001124929FA001939F500D112470E0CA01BE
:102C30000E9450266038710540F46115710519F441
:102C400006C068E070E0862F08958FE7089581E060
:102C5000089580919C0280FF08C06091050170E09A
:102C6000759567957595679521C081FF06C0609140
:102C7000050170E07595679519C082FF04C06091E9
:102C8000050170E010C090919A02992399F060912B
:102C900004019617A0F780910501899FC0011124B6
:102CA00070E00E9450266038710540F4611571058E
:102CB00019F406C061E070E0862F08958FE708954B
:102CC00081E008958D3E21F40E94EA15819504C0AB
:102CD0008E3E29F40E94EA158093A00208958F3E4B
:102CE00021F40E94EA15819504C0803F29F40E94D6
:102CF000EA1580939F020895893F19F40E942916CE
:102D000005C08A3F31F40E94291681958093A10263
:102D100008958B3F21F40E942916819504C08C3FB1
:102D200029F40E9429168093A20208959FE0980F2B
:102D3000983078F421E030E0A90102C0440F551F1B
:102D40009A95E2F7CA0190919E02892B80939E0288
:102D500008958D3F21F480919C0281600BC08E3FCD
:102D600021F480919C02826005C08F3F29F48091FC
:102D70009C02846080939C0208958D3E39F490916A
:102D8000A00297FF35C01092A00259C08E3E29F4D0
:102D90009091A0021916BCF32BC090919F028F3E18
:102DA00029F497FF25C010929F0249C0803F19F473
:102DB0001916CCF31DC09091A102893F29F4191670
:102DC000BCF41092A1023BC08A3F19F497FF10C0D7
:102DD000F8CF8B3F39F49091A20297FF09C010926F
:102DE000A2022DC08C3F21F49091A2021916BCF3CF
:102DF0009FE0980F983080F421E030E0A90102C0F4
:102E0000440F551F9A95E2F7CA01809590919E0252
:102E1000892380939E0213C08D3F21F480919C02F0
:102E20008E7F0BC08E3F21F480919C028D7F05C068
:102E30008F3F29F480919C028B7F80939C0280912C
:102E40009F02811106C08091A002811102C01092E0
:102E50009B028091A102811106C08091A202811182
:102E600002C010929A0208950E94DC1E20919F02D7
:102E7000211104C02091A002222321F090939902F5
:102E8000809398022091A102211104C02091A202F6
:102E9000222321F090939702809396028DE992E08D
:102EA0000C94481DEF92FF920F931F93CF93DF93E3
:102EB00000D000D000D0CDB7DEB786E0EDE9F2E07B
:102EC000DE01119601900D928A95E1F7E0909F0244
:102ED000F090A0020091A1021091A20210929F0214
:102EE0001092A0021092A1021092A202E11003C05F
:102EF000FF2009F45DC080919802909199020E9490
:102F0000F41EAC0190919B02992339F020910901A4
:102F100030E02417350758F04BC0209195028AE025
:102F2000289F900111242417350718F041C09F3FB6
:102F300019F09F5F90939B02EE2061F00E94EA15CA
:102F40001E1414F09FEF01C091E0989F902D112462
:102F500090939F02FF2061F00E94EA151F1414F065
:102F60009FEF01C091E0989F902D11249093A002B3
:102F700030919F023323E1F02091A0022223C1F07F
:102F800045EB3403C0011124992319F090939F025B
:102F900003C081E080939F0235EB2303C00111241D
:102FA000992319F09093A00203C081E08093A002BE
:102FB000011103C0112309F45DC080919602909124
:102FC00097020E94F41EAC0190919A02992339F065
:102FD0002091060130E02417350758F04BC02091AE
:102FE00094028AE0289F900111242417350718F0D5
:102FF00041C09F3F19F09F5F90939A02002361F0B8
:103000000E942916101614F09FEF01C091E0989FBE
:10301000902D11249093A102112361F00E94291692
:10302000111614F09FEF01C091E0989F902D11248C
:103030009093A2023091A1023323E1F02091A202E9
:103040002223C1F045EB3403C0011124992319F068
:103050009093A10203C081E08093A10235EB23038A
:10306000C0011124992319F09093A20203C081E0BA
:103070008093A20280919F0281110BC08091A002D7
:10308000811107C08091A102811103C08091A20229
:1030900081110E943417EB82FC820D831E8386E02F
:1030A000FE013196ADE9B2E001900D928A95E1F70B
:1030B00026960FB6F894DEBF0FBECDBFDF91CF913D
:1030C0001F910F91FF90EF900895EDE9F2E086E0F7
:1030D000DF011D928A95E9F710929B0210929A02E5
:1030E00010929C020895CF93DF9397FF0DC0FB01D0
:1030F0002281222349F0EC010E94B118CE019F7772
:103100000E9424190E94FE1881E0DF91CF9108955A
:103110009091D902923069F48A3040F490E0099697
:103120006AE070E00E945026875A01C086500C94D5
:1031300070080C94DB068CE090E00E94772690E00B
:10314000A0E0B0E08093D9029093DA02A093DB0272
:10315000B093DC0208956091D9028CE090E00C9469
:1031600085260E942B1D869581708093DE020E9429
:103170002B1D81708093D8028091D902813039F45F
:103180008091DE02882319F089E30E9470080E9472
:1031900029118093DD020E943C118091D902813077
:1031A00071F048F0823081F0843009F586EE0E949B
:1031B000700888E11AC082EE0E94CF0718C088E12B
:1031C00093E00E942A0513C08091D802811103C0A8
:1031D00083E50E94700882EE0E94CF078FE39CE98E
:1031E0000197F1F700C0000087E50E9470088FE3A7
:1031F0009CE90197F1F700C0000008958091D90281
:10320000813059F030F0823089F08430C9F488E29E
:1032100015C082EE0E94250813C08CE20E9470083F
:103220008091DE02882361F089E308C082EE0E946B
:1032300025088091D802811103C083E50E9470089F
:103240008091DD020C9439110F931F93CF93DF937C
:103250008C01CCE0D0E0C8010C2E02C09695879579
:103260000A94E2F78F700E9488182497CC3F8FEF62
:10327000D80789F7DF91CF911F910F9108950F9390
:103280001F93CF93DF93EC018B01FB018281882395
:1032900061F00E942911CE01825E9C458530910526
:1032A00020F48093D9020E94AB18B801CE01DF91BF
:1032B000CF911F910F910C947318CF93DF93EC0172
:1032C000FB018281882309F43CC1C430FDE5DF079E
:1032D00060F4CB3F9CE5D90788F49E0122503C4521
:1032E0002431310508F02EC109C0C236EDE5DE07F4
:1032F00029F0C63AFDE5DF0709F024C10E94221239
:103300009093D7028093D602C1318CE5D80709F497
:10331000C6C008F042C0C930ECE5DE0709F49BC026
:1033200000F5C5308CE5D80709F485C078F4C330C2
:10333000ECE5DE0709F478C008F07AC0C230DC455D
:1033400009F0F5C08091D6028160EFC0C7309CE5DE
:10335000D90709F478C008F07AC08091D60280615C
:10336000E4C0CD30FCE5DF0709F487C058F4CB306A
:103370009CE5D90709F479C008F07BC08091D6029A
:1033800088606FC0CF30FCE5DF0709F480C008F02B
:1033900082C08091D602877FC8C0CE3F9CE5D90706
:1033A00009F471C000F5C531FCE5DF0709F485C0FB
:1033B00068F4C3319CE5D90709F475C008F095C0DD
:1033C0000E94AE0B8091D6028F77AFC0CC3FFCE558
:1033D000DF07A9F108F054C0CB3FDC4509F0A7C0D6
:1033E0008091D70240C0C230EDE5DE0709F489C004
:1033F00058F4C1158DE5D80709F45AC008F069C022
:103400008091D70282602FC0C236EDE5DE0709F455
:103410007CC0C63AFDE5DF0709F481C0C330DD4555
:1034200009F085C080E06EC08091D60282607DC0C8
:103430008091D60216C08091D602886076C08091B5
:10344000D70282604FC08091D60280626EC08091A8
:10345000D60280646AC00E94AE0B8091D60280685A
:1034600064C0846062C081603DC08091D6028E7F5E
:103470005CC08091D6028D7F58C08091D60216C064
:103480008091D70218C08091D7028D7F2BC0809188
:10349000D6028F7E4AC08091D6028F7D46C0809131
:1034A000D6028F7B42C08091D602877F8B7F3DC042
:1034B0008091D7028D7F8E7F15C08091D60282FBCE
:1034C000222720F991E0922790FB82F990FB83F963
:1034D0002CC08091D702982F909591708E7F892B68
:1034E00090FB81F98093D70222C00E94AE0B80919D
:1034F000D60287FB222720F991E0922790FB87F9DB
:1035000014C081E00E94B91212C08091D60284FBDF
:10351000222720F991E0922790FB84F906C0809140
:10352000D602982F909590FB80F98093D6028091D7
:10353000D6029091D7020E9433120E94AE0B80E017
:1035400001C081E0DF91CF910895CF93DF93863161
:103550009C4541F5EB010E942911982F8A81209109
:10356000020130910301882379F09A7A81E009F40D
:1035700080E08093A302911102C069E201C065E37B
:10358000C9010E94181E0AC08091A302811102C0C5
:1035900069E201C065E3C9010E94231E0E946E1109
:1035A00080E001C081E0DF91CF9108950F931F93D8
:1035B000CF93DF93C42FD22FFC0182818823C9F0DF
:1035C0004093A6020E94DC1E9093A5028093A40261
:1035D00080E28C0F883008F057C0C77081E001C0CE
:1035E000880FCA95EAF7DF91CF911F910F910C9444
:1035F00079088091A602481330C08091A40290916E
:10360000A5020E94F41E883C910538F510E21D0FBA
:10361000CD17B9F080E28C0F883040F4C77081E09C
:1036200001C0880FCA95EAF70E948008183028F573
:1036300081E09D2F977001C0880F9A95EAF70E944C
:103640007908802F0E9470081830F0F4D77081E05C
:1036500001C0880FDA95EAF70AC080E28C0F883043
:1036600098F4C77081E001C0880FCA95EAF7DF912E
:10367000CF911F910F910C948008802FDF91CF91F3
:103680001F910F910C947008DF91CF911F910F91B2
:1036900008950F939C01CB01243F4CE5340731F191
:1036A00088F4293DFCE53F07D9F02A3D4CE5340775
:1036B00079F1283D3C45A9F506E221EE41EE68EDA1
:1036C0007CE52BC0263FFCE53F07E1F0A8F0273F53
:1036D0003C4539F507E225EE46EE67EF7CE51DC077
:1036E00007E225EE45EE69ED7CE517C006E221EE26
:1036F00040EE64EF7CE511C007E225EE44EE65EF95
:103700007CE50BC006E221EE42EE66EF7CE505C0EB
:1037100008E221E045EE6AED7CE50E94D61A80E0E1
:1037200008C0FC018281882319F01092A60201C012
:1037300081E00F9108951092B9008CE08093B80059
:1037400008959F92AF92BF92CF92DF92EF92FF9235
:103750000F931F93CF93DF93B82EEB010E94DC1ED3
:103760006C01C431D10558F0CF3F8FEFD80759F025
:10377000CE0164E170E00E943C267B0107C0EE248C
:10378000E394F12C03C025E0E22EF12C84E8A82E6E
:1037900094EA992E1092BC009092BC000E94DC1E0C
:1037A0008C018091BC0087FD08C00E94DC1E801B3C
:1037B000910B8E159F05A8F32AC08091B900887FD0
:1037C000883041F08091B900887F803119F00FEF87
:1037D0001FEF1FC0B092BB00A092BC000E94DC1E75
:1037E0008C018091BC0087FD08C00E94DC1E801BFC
:1037F000910B8E159F05A8F30AC08091B900887FB0
:10380000883111F0803419F700E010E00EC00EEF9F
:103810001FEFCF3F8FEFD80709F4BCCFC6010E943E
:10382000F41E8C179D0708F4B5CFC801DF91CF9126
:103830001F910F91FF90EF90DF90CF90BF90AF90CE
:103840009F9008950F931F93CF93DF93EB01809385
:10385000BB0084E88093BC000E94DC1E8C01809138
:10386000BC0087FD0EC0CF3F8FEFD807C1F30E9489
:10387000DC1E801B910B8C179D0788F38EEF9FEF4A
:103880000CC02091B900287F81E090E0283211F42B
:1038900080E090E0919581959109DF91CF911F9102
:1038A0000F9108950F931F93CF93DF93EC0184EC56
:1038B0008093BC000E94DC1E8C018091BC0087FDBF
:1038C0000EC0CF3F8FEFD807C1F30E94DC1E801BD4
:1038D000910B8C179D0788F38EEF9FEF03C08091AB
:1038E000BB0090E0DF91CF911F910F9108950F934E
:1038F0001F93CF93DF93EC0184E88093BC000E9478
:10390000DC1E8C018091BC0087FD0EC0CF3F8FEF85
:10391000D807C1F30E94DC1E801B910B8C179D07FA
:1039200088F38EEF9FEF03C08091BB0090E0DF91A2
:10393000CF911F910F910895CF92DF92EF92FF9256
:103940000F931F93CF93DF93C62F6A017901B801BC
:103950000E94A11B97FD11C0B8018C2F0E94221C50
:10396000E601EC0CFD1CCE15DF0539F097FD05C016
:10397000B80189910E94221CF6CF24E92093BC0053
:10398000DF91CF911F910F91FF90EF90DF90CF903B
:103990000895CF92DF92EF92FF920F931F93CF93F0
:1039A000DF93D82EC62E7A01E901B8010E94A11B2F
:1039B00097FD2AC0B8018C2D0E94221C97FD24C0BF
:1039C000B8018D2D81600E94A11B6701219796018E
:1039D0002E193F092C173D0768F497FD15C0C80143
:1039E0000E94521C97FD02C0F6018083FFEFCF1AA0
:1039F000DF0AEDCF97FD08C0C8010E94771C97FD34
:103A000003C0CE0DDF1D888324E92093BC00181667
:103A1000190614F480E090E0DF91CF911F910F918F
:103A2000FF90EF90DF90CF90089590939F01809347
:103A30009E0108959093AC028093AB020895E091AB
:103A4000AB02F091AC02309721F00190F081E02DB3
:103A5000099480E008950E941F1D0895E091AB0233
:103A6000F091AC02309799F020911601222359F081
:103A70002091D60227FF07C0DC012C9111962C93D0
:103A8000119726E02C930280F381E02D099408958C
:103A9000E091AB02F091AC02309739F022E0DC010A
:103AA0002C930480F581E02D099408952091A902BA
:103AB0003091AA022817390771F09093AA028093D7
:103AC000A902E091AB02F091AC02309721F00680A0
:103AD000F781E02D099408952091A7023091A80262
:103AE0002817390771F09093A8028093A702E091FC
:103AF000AB02F091AC02309721F00084F185E02D0B
:103B000009940895FC01329680911601882331F0C2
:103B10008091D60287FF02C09EE101C096E080E05E
:103B2000915028F021912223D9F38F5FF9CF089586
:103B3000662351F1209116012223E9F02091D6024B
:103B400027FF19C0462F4695469546954E31E0F41D
:103B5000677021E030E002C0220F331F6A95E2F760
:103B6000FC01E40FF11D828190E02823392381E0DC
:103B7000232B69F409C0FC01329608962191621743
:103B800029F0E817F907D1F780E0089581E008955A
:103B90009C01FC0132969FEF80E04191461789F02D
:103BA0009F3F19F4411101C0982F8F5F8630A9F70C
:103BB0009F3F39F0F901E90FF11D97FDFA956283F6
:103BC000089508959C012A5F3F4FFC0142814613EE
:103BD00001C01282019682179307B9F70895262F24
:103BE0002695269526952E3168F4FC01E20FF11DED
:103BF000677021E030E001C0220F6A95EAF7828108
:103C0000282B22830895262F2695269526952E313A
:103C100070F4FC01E20FF11D677021E030E001C09B
:103C2000220F6A95EAF7209582812823228308953E
:103C300020911601222329F02091D60227FD0C9411
:103C4000EF1D0C94C81D20911601222329F020910C
:103C5000D60227FD0C94031E0C94E21D2091160140
:103C6000FC013296222331F08091D60287FF02C0F8
:103C70008EE101C086E0DF011D928A95E9F7089583
:103C800008950C94401E83E08093AD020C94411E75
:103C9000811102C081E001C082E08093AD020C94EA
:103CA000411E0C94481E81E08093AD020C94411E8D
:103CB0000C94531E08950C945A1E0C945B1E0C9485
:103CC0005A1E0C945A1E0C945A1ECF930E94611EC9
:103CD0000E948E030E945F1EC0E08C2F0E94AF04E2
:103CE000892B29F4CF5FC630C1F780E001C081E0A5
:103CF000CF91089508951F920F920FB60F9211243D
:103D00008F939F93AF93BF938091AE02811113C0A5
:103D10008091DF029091E002A091E102B091E20275
:103D20004196A11DB11D8093DF029093E002A09304
:103D3000E102B093E202BF91AF919F918F910F90FA
:103D40000FBE0F901F9018958091E702843031F1DB
:103D50000E94FD051092AE0220E488E190E00FB6CB
:103D6000F894A895809360000FBE2093600083B7FD
:103D7000817F846083BF83B7816083BF7894889597
:103D800083B78E7F83BF0FB6F894A89580916000AB
:103D9000886180936000109260000FBE08950E94B9
:103DA000AE0B0C94010682E084BD93E095BD9AEFC2
:103DB00097BD80936E0008952FB7F8948091DF022D
:103DC0009091E002A091E102B091E2022FBF08952C
:103DD0002FB7F8946091DF027091E0028091E102C8
:103DE0009091E2022FBF08959C014FB7F894809103
:103DF000DF029091E002A091E102B091E2024FBF98
:103E0000821B930B089578941F920F920FB60F9216
:103E100011248F939F93AF93BF938091DF02909172
:103E2000E002A091E102B091E2020196A11DB11D54
:103E30008093DF029093E002A093E102B093E2024C
:103E4000BF91AF919F918F910F900FBE0F901F90D8
:103E50001895F89481E08093E00080E28093D80088
:103E6000E9ECF0E010828FE19EE40197F1F700C0E9
:103E700000001DBA109268001CBC10BE1FBA109240
:103E80007A0010926E0010926F00109271001092E2
:103E900072001082ECEBF0E0108214B817B81AB878
:103EA0001DB810BA108215B818B81BB81EB811BAD0
:103EB0000C94003F08958091D2020895089522E065
:103EC0002093E9002FEF3091E800215035FD06C026
:103ED00035ED3A95F1F700002111F5CF2091E8007A
:103EE00025FF0BC040E050E066E070E00E949E219C
:103EF0008091E8008E778093E8000895CF93DF9358
:103F000020911601222339F02091D60227FF03C009
:103F100060E222E002C068E021E02093E9002FEF98
:103F20003091E800215035FD06C035ED3A95F1F7A6
:103F300000002111F5CF2091E80025FF1DC0EC0104
:103F400080911601811105C040E050E068E070E00A
:103F500003C070E040E050E0CE010E949E218091BD
:103F6000E8008E778093E80080E2FE01A2EBB2E0E9
:103F700001900D928A95E1F7DF91CF91089580939A
:103F8000AF027093B1026093B0028091E702843077
:103F900001F582E08093E9008FEF9091E800815075
:103FA00095FD06C095ED9A95F1F700008111F5CFCA
:103FB0008091E80085FF0DC040E050E063E070E0D4
:103FC0008FEA92E00E949E218091E8008E77809394
:103FD000E8000895BC0184E00C94BF1FBC0183E09D
:103FE0000C94BF1F8091E602811109C00E942F230B
:103FF0000E948C238091E20084608093E200089507
:104000001092E60208950C94581E6091E30281E03C
:10401000611101C080E00C94431E9091E70281E0A1
:10402000943009F080E06091E3020C94481E42E075
:1040300061EC81E00E94A82242E261EC82E00E94F1
:10404000A8229091E70281E0943009F080E060912D
:10405000E3020C94511E8091E902833009F461C09F
:1040600030F4813071F0823009F49AC008958A30BA
:1040700009F486C08B3009F46CC0893009F0A8C0FF
:1040800020C08091E802813A09F0A2C08091E80046
:10409000877F8093E8008091EC029091ED02892B5C
:1040A00021F460E282EB92E003C060E080E090E007
:1040B00070E00E94E9218091E8008B778093E8000E
:1040C00008958091E802813209F082C08091EC026B
:1040D0009091ED02029708F07BC08091E800877F05
:1040E0008093E8008091E80082FD05C08091E7029E
:1040F0008111F8CF6DC02091F3008091F20090E023
:10410000922B029731F48091F100813011F08630CA
:1041100021F48091F1008093D2028091E8008B77A6
:1041200053C08091E802813A09F052C08091EC02BC
:104130009091ED02892B09F04BC08091E800877FB8
:104140008093E8008091E80080FFFCCF8091160109
:1041500036C08091E8028132D9F58091EC029091CD
:10416000ED02892BA9F58091E800877F8093E80014
:104170000E94DD228091EA02809316010C94AE0B1E
:104180008091E802813221F58091E800877F809359
:10419000E8000E94DD228091EB028093D302089513
:1041A0008091E802813AA1F48091E800877F8093B2
:1041B000E8008091E80080FFFCCF8091D3028093DB
:1041C000F1008091E8008E778093E8000C94DD2266
:1041D000089584B7877F84BF0FB6F894A89580911F
:1041E0006000886180936000109260000FBE90E0D4
:1041F00080E80FB6F89480936100909361000FBE41
:104200000C94531E0E942F230E948C23E2EEF0E0B8
:1042100080818460808378940C9421268AE091E0E8
:104220000C941A1D8091E7028530A9F48091E70271
:10423000853079F40E94A41E8091E5028823B1F3B1
:104240000E94651E882391F30E9488210E94AE0B74
:10425000EDCF0C94CF1E089508950C942F21292F93
:10426000332723303105C9F060F42130310581F066
:104270002230310509F044C08BE390E02AE234E0BB
:1042800043C021323105E1F02232310549F138C015
:1042900082E190E025E634E037C09927813091052E
:1042A00049F028F0029761F5E4E0F4E005C0E6E2A9
:1042B000F4E002C0E4E1F4E0849190E09F0124C0C6
:1042C0006115710541F061307105D1F489E090E02C
:1042D00025E534E019C089E090E02CE334E014C017
:1042E0006115710541F06130710551F486EB90E084
:1042F00027E734E009C080E490E02DE235E004C017
:1043000080E090E020E030E0FA01318320830895DE
:1043100080E189BD82E189BD09B400FEFDCF8091B5
:10432000D8008F7D8093D8008091E00082608093D8
:10433000E0008091E00081FDFCCF0895CF92DF92F4
:10434000EF92FF920F931F93CF93DF93EC018B01BA
:104350007A010E94FC22811133C0E114F10439F08A
:10436000F70180819181081B190BC80FD91FC12C3F
:10437000D12C0115110519F18091E80085FD16C0B9
:104380008091E8008E778093E800E114F10449F011
:10439000F70180819181C80ED91ED182C08285E04B
:1043A0000FC00E94FC22882321F30AC089918093C8
:1043B000F10001501109FFEFCF1ADF0ADACF80E0D8
:1043C000DF91CF911F910F91FF90EF90DF90CF90F1
:1043D00008952091EE023091EF022617370748F03A
:1043E0006115710539F42091E8002E772093E800DB
:1043F00001C0B901FC0120E06115710579F18091DE
:10440000E7028823F1F18530F1F18091E80083FD26
:104410003CC08091E80082FD2EC08091E80080FFC2
:10442000EBCF2091F3008091F20090E0922B611588
:10443000710551F08830910538F421912093F100F5
:10444000615071090196F3CF21E0089709F020E04F
:104450008091E8008E778093E800CECF2111CFCFF6
:104460000AC08091E702882361F0853061F0809175
:10447000E80083FD0AC08091E80082FFF2CF80E06F
:10448000089582E0089583E0089581E008952091E1
:10449000EE023091EF022617370748F061157105DB
:1044A00039F42091E8002E772093E80001C0B9018B
:1044B000FC0120E06115710591F18091E7028823EC
:1044C00009F440C0853009F43FC08091E80083FDC5
:1044D0003DC08091E80082FD2FC08091E80080FF00
:1044E000E9CF2091F3008091F20090E0922B6115CA
:1044F000710559F08830910540F424912093F10022
:104500003196615071090196F2CF21E0089709F0C8
:1045100020E08091E8008E778093E800CBCF2111D6
:10452000CCCF0AC08091E702882361F0853061F02A
:104530008091E80083FD0AC08091E80082FFF2CFFD
:1045400080E0089582E0089583E0089581E0089571
:10455000982F973068F59093E900981739F070918B
:10456000EC002091ED005091F00003C0242F762F35
:1045700050E021FD02C09F5FECCF3091EB003E7F09
:104580003093EB003091ED003D7F3093ED003091A2
:10459000EB0031603093EB007093EC002093ED0062
:1045A0005093F0002091EE0027FDE5CF80E00895C4
:1045B0008F708093E90081E008958091E80287FF81
:1045C00011C08091E80082FD05C08091E702811151
:1045D000F8CF11C08091E8008B770BC08091E70283
:1045E000882349F08091E80080FFF8CF8091E800AF
:1045F0008E778093E80008952091E4003091E500E3
:1046000095E64091EC00842F817040FF23C080919B
:10461000E80080FD1DC08091E702882399F0853075
:1046200099F08091EB0085FD11C04091E40050911C
:10463000E5002417350729F3915011F09A01E1CFD5
:1046400084E0089582E0089583E0089581E008956C
:1046500080E008954091E80042FFDDCF08950E9478
:104660009D230E94A523E0EEF0E08081816080839D
:10467000E8EDF0E080818F77808319BCA7EDB0E092
:104680008C918E7F8C9380818F7E80831092E60246
:1046900008950F931F93CF93DF930E949D230E9451
:1046A000A523C8EDD0E088818F77888388818068D2
:1046B000888388818F7D888319BC1092E7021092CD
:1046C000E3021092E5021092E40200EE10E0F8011D
:1046D00080818B7F808388818160888342E060E075
:1046E00080E00E94A822E1EEF0E080818E7F80834E
:1046F000E2EEF0E080818160808380818860808349
:10470000F80180818E7F8083888180618883DF913A
:10471000CF911F910F910895E8EDF0E080818F7E99
:104720008083E7EDF0E080818160808384E082BF58
:1047300081E08093E6020C944923E8EDF0E080816B
:104740008E7F80831092E20008951092DA0010921A
:10475000E10008951F920F920FB60F9211242F932C
:104760003F934F935F936F937F938F939F93AF93F9
:10477000BF93EF93FF938091E10082FF0BC0809184
:10478000E20082FF07C08091E1008B7F8093E1000F
:104790000E9420268091DA0080FF1FC08091D800FF
:1047A00080FF1BC08091DA008E7F8093DA008091B9
:1047B000D90080FF0DC080E189BD82E189BD09B4C7
:1047C00000FEFDCF81E08093E7020E94F21F05C04A
:1047D00019BC1092E7020E9400208091E10080FF46
:1047E00019C08091E20080FF15C08091E2008E7FA9
:1047F0008093E2008091E20080618093E2008091EA
:10480000D80080628093D80019BC85E08093E702CD
:104810000E9405208091E10084FF30C08091E20079
:1048200084FF2CC080E189BD82E189BD09B400FE0E
:10483000FDCF8091D8008F7D8093D8008091E100DA
:104840008F7E8093E1008091E2008F7E8093E20072
:104850008091E20081608093E2008091E3028823EE
:1048600011F084E007C08091E30087FD02C081E081
:1048700001C083E08093E7020E940D208091E10057
:1048800083FF29C08091E20083FF25C08091E10071
:10489000877F8093E10082E08093E7021092E30239
:1048A0008091E1008E7F8093E1008091E2008E7F15
:1048B0008093E2008091E20080618093E20042E018
:1048C00060E080E00E94A8228091F00088608093E0
:1048D000F0000E940320FF91EF91BF91AF919F9153
:1048E0008F917F916F915F914F913F912F910F9099
:1048F0000FBE0F901F9018951F920F920FB60F9238
:1049000011242F933F934F935F936F937F938F93D4
:104910009F93AF93BF93CF93DF93EF93FF93C09198
:10492000E900CF708091EC00D82FD17080FDD0E8E5
:104930001092E9008091F000877F8093F0007894D6
:104940000E94C0241092E9008091F000886080935A
:10495000F000CD2BCF70C093E900FF91EF91DF9174
:10496000CF91BF91AF919F918F917F916F915F9107
:104970004F913F912F910F900FBE0F901F90189560
:104980001F93CF93DF93CDB7DEB7AA970FB6F894F6
:10499000DEBF0FBECDBFE8EEF2E08091F100819363
:1049A00022E0E03FF207C9F70E942B208091E80047
:1049B00083FF2EC18091E8029091E902492F50E0D7
:1049C0004A30510508F024C1FA01E759FF4F0C9411
:1049D0006426803821F0823809F01AC108C080911D
:1049E000E4029091E502992389F082600FC08091E2
:1049F000EC028F70873008F00BC18093E900809142
:104A0000EB0085FB882780F91092E9009091E8007F
:104A1000977F9093E8008093F1001092F100D1C04D
:104A2000282F2D7F09F0F4C0882319F0823061F01F
:104A3000EFC08091EA02813009F0EAC0933009F0BA
:104A400080E08093E5022EC08091EA0281112AC0A5
:104A50008091EC028F702FEF280F263008F0D8C01D
:104A60008093E9002091EB0020FF1CC0933021F4DB
:104A70008091EB00806214C09091EB009061909364
:104A8000EB0021E030E0A90102C0440F551F8A95D8
:104A9000E2F74093EA001092EA008091EB00886010
:104AA0008093EB001092E9008091E800877F80936B
:104AB000E8000E94DD22ACC08111AAC01091EA0278
:104AC0001F778091E3008078812B8093E3008091B1
:104AD000E800877F8093E8000E94DD228091E80053
:104AE00080FFFCCF8091E30080688093E300111188
:104AF00002C082E001C083E08093E70289C0805851
:104B0000823008F085C08091EA029091EB028C3DE2
:104B100053E0950779F583E08A838AE289834FB76A
:104B2000F894DE01139620E03EE051E2E32FF0E03E
:104B300050935700E49120FF03C0E295EF703F5F70
:104B4000EF708E2F90E0EA3010F0C79601C0C0964B
:104B50008D939D932F5F243149F74FBF8091E800DB
:104B6000877F8093E8006AE270E0CE0101960E94A0
:104B7000E92116C06091EC027091ED02AE014F5F29
:104B80005F4F0E942D21BC01892B09F441C09091F7
:104B9000E800977F9093E80089819A810E944722DC
:104BA0008091E8008B778093E80032C0803881F5EF
:104BB0008091E800877F8093E8008091E3028093F2
:104BC000F1008091E8008E7772CF811121C0809131
:104BD000EA029091EB0299270297D4F48091E800C1
:104BE000877F8093E8008091EA028093E3020E942D
:104BF000DD228091E302811106C08091E30087FDF0
:104C000002C081E001C084E08093E7020E94172087
:104C10008091E80083FF0AC08091E800877F80933D
:104C2000E8008091EB0080628093EB00AA960FB6BB
:104C3000F894DEBF0FBECDBFDF91CF911F910895D5
:104C40000895CF938091E7028823A1F0C091E900F5
:104C5000CF709091EC00892F817090FD80E8C82B77
:104C60001092E9008091E80083FD0E94C024CF707B
:104C7000C093E900CF910895AA1BBB1B51E107C067
:104C8000AA1FBB1FA617B70710F0A61BB70B881FDC
:104C9000991F5A95A9F780959095BC01CD0108956B
:104CA00097FB072E16F4009407D077FD09D00E94D9
:104CB0003C2607FC05D03EF4909581959F4F0895C2
:104CC000709561957F4F0895EE0FFF1F0590F49149
:104CD000E02D0994FB01DC0104C08D910190801945
:104CE00021F441505040C8F7881B990B0895F99959
:104CF000FECF92BD81BDF89A992780B50895A8E1AD
:104D0000B0E042E050E00C94AB26262FF999FECF9C
:104D100092BD81BDF89A019700B4021639F01FBA0E
:104D200020BD0FB6F894FA9AF99A0FBE089503962B
:104D3000272F0E9486260E948526252F0E948626E0
:104D4000242F0C9486260196272F0E9486260C94E9
:104D50008526DC01CB01FC01F999FECF06C0F2BD2E
:104D6000E1BDF89A319600B40D9241505040B8F729
:064D70000895F894FFCF46
:104D7600C8005D022808503C07145B1F7E1F5F1F9A
:104D8600EE1FEA1F5E1F0100010203040501010177
:104D960001010100000000000000000000000031D9
:104DA6003233929366F0F1F4F5F6F7E200E900EAA1
:104DB60000B500B600B700CD008301CC008A019291
:104DC6000194012102230224022502260227022A37
:104DD60002B300B4006F007000818283E200E90034
:104DE600EA00B500B600B700CD008301CC008A0109
:104DF600920194012102230224022502260227029F
:0E4E06002A02B300B4006F00700081828300A6
:00000001FF
